:0200000480007A
:1000000037F1FF7FEF00600873000000B68B3A8C79
:10001000BE8C428D0A8FAA83054563597500130172
:1000200001802A836B5003000505C5BF7A81014515
:10003000B28F9E8DEBE0BF01170500001305053A56
:100040006B400500B708010023A0B80082801703A9
:1000500000001303E3FB6B0003008280511106C014
:100060002EC28345050081C5F13F0505DDBF8240F5
:10007000924531018280511106C02EC293050503BD
:10008000D1378240924531018280011106CE22CCC7
:100090000010232604FE15A80327C4FEBA878E0786
:1000A000998F8A07998F139747001D8F9317270001
:1000B0003E87B707008193874724BA973E85912AE8
:1000C0008327C4FE85072326F4FE0327C4FE9D472D
:1000D000E3D4E7FCB70700819387871F37070081C8
:1000E00013078717B70600819386861337060080AB
:1000F00013064617A145094541210945A12BB7071C
:10010000008113850704993FB70700811385C70550
:10011000B137232404FE3DA8832784FE3E852D2489
:10012000B707008113858706153FB70700810327AE
:1001300084FE0A079387871FBA979C433E8529242C
:10014000B70700811385C706113F832784FE850703
:100150002324F4FE032784FEBD47E3DFE7FAB70755
:10016000008113850707DD3D81473E85F2406244EB
:1001700005618280397106DE22DC80002326A4FC22
:100180002324B4FC99232326A4FE912B2324A4FE2C
:100190008D232322A4FE832784FC8E070327C4FC1F
:1001A000BA972320F4FE832704FE93B7B70093C7C2
:1001B0001700A30FF4FC8347F4FD3E8FB7070080C0
:1001C000938F27206B200F007B70FF01832704FE95
:1001D0008A070327C4FEBA979443832704FE8A073D
:1001E000032784FEBA979843832704FE8A070326D1
:1001F00044FEB297369798C3B7070080138E472006
:10020000028E01006B3000000100F2506254216147
:100210008280AA8201439D4323A0620023A2620040
:1002200023A4620023A6720023A862008280AA820F
:1002300003A38200050323A462001383420183AE5B
:10024000420093935E001E9303AE05002320C3017A
:1002500003AE45002322C30103AE85002324C3015E
:1002600003AEC5002326C30103AE05012328C30145
:1002700003AE4501232AC30103AE8501232CC3012C
:1002800003AEC501232EC301850E130F2003639413
:10029000EE01930E000023A2D2018280AA8203A362
:1002A00082007D1323A462001383420183AE020007
:1002B000930F2003768F050F6314FF01130F0000C7
:1002C00023A0E20193935E001E93032E030023A05C
:1002D000C501032E430023A2C501032E830023A4DE
:1002E000C501032EC30023A6C501032E030123A8C5
:1002F000C501032E430123AAC501032E830123ACAC
:10030000C501032EC30123AEC5018280AA8203A3C7
:10031000820013050000130E200363136E00050511
:100320008280AA8203A3820013050000130E00003E
:1003300063136E0005058280AA8203A3C20083A313
:10034000020133B563008280797106D622D4001889
:10035000232EA4FC0327C4FDBD4763EEE700B707C7
:1003600000810327C4FD0A079387871BBA979C4324
:100370003E85ED31B1A8930700022326F4FEA305C4
:1003800004FE8327C4FEF1170327C4FDB357F7000B
:10039000BD8B2322F4FE832744FE81C78547A30536
:1003A000F4FE8347B4FE81CFB7070081032744FEE4
:1003B0000A079387871BBA979C433E85453183275D
:1003C000C4FEF1172326F4FE8327C4FEE34BF0FAA4
:1003D000B250225445618280797106D622D46AD205
:1003E00000186A87BA878E07998F8A07998F1397A3
:1003F00047001D8F931727003E87B707008193871B
:100400004724BA973E85313FAA878DCBB707008135
:100410001385470DA131EA873E853D37B707008137
:100420001385C70D25396A87B73700819387474EF3
:10043000BA9705472380E700730000006A87BA87F0
:100440008E07998F8A07998F139747001D8F9317EF
:1004500027003E87B707008193874724BA97130781
:1004600004FDBA853E851D3D832784FD3E8103251D
:1004700044FD832504FD0326C4FD832604FE0327D3
:1004800044FE832784FE0328C4FE4936730000001F
:100490000100B2502254125D45618280397106DE3E
:1004A00022DC80008A89232604FE69A00327C4FE7B
:1004B000BA878E07998F8A07998F139747001D8FE8
:1004C000931727003E87B707008193874724BA9781
:1004D0003E85813DAA87B1EB0327C4FEBA878E070C
:1004E000998F8A07998F139747001D8F93172700BD
:1004F0003E87B707008193874724BA971307C4FC48
:10050000BA853E85613B832744FD3E81032504FD7A
:100510008325C4FC032684FD8326C4FD032704FE33
:10052000832744FE032884FE1D368327C4FE8507E7
:100530002326F4FE0327C4FE9947E3D9E7F64E814C
:100540000100F250625421618280797122D6001834
:10055000232EA4FC232604FE31A08327C4FE850796
:100560002326F4FE0327C4FE8327C4FDE347F7FEDA
:1005700001003254456182801D7186CEA2CC80106C
:10058000232EA4FA232CB4FA232AC4FA2328D4FA5B
:100590002326E4FA2324F4FA13090100232604FE97
:1005A000232404FE51A8C1794E91832784FE23247D
:1005B000F4FC832784FB2326F4FC8A872328F4FC9D
:1005C000832744FB232AF4FC832704FB232CF4FC1D
:1005D0008327C4FA232EF4FC832784FA2320F4FE15
:1005E0008327C4FE2322F4FE0327C4FEBA878E07A6
:1005F000998F8A07998F139747001D8F93172700AC
:100600003E87B707008193874724BA97130784FC76
:10061000BA853E8529398327C4FE85072326F4FE43
:100620000327C4FE994763D4E700232604FE8327EB
:1006300084FE85072324F4FE032784FE8327C4FB5E
:10064000E363F7F613010900913D0100F6406644AB
:1006500025618280797106D622D40018232EA4FC4D
:10066000B70700811385070ED53AA30704FE91A0B2
:100670008547A307F4FE232404FE35A08347F4FE38
:10068000373700819306474E032784FE369703478A
:100690000700F98FB337F000A307F4FE832784FE29
:1006A00085072324F4FE832784FE0327C4FDE3E7A4
:1006B000E7FC8347F4FE93C7170093F7F70FCDFBD2
:1006C0000100B250225445618280411122C65EC4AD
:1006D0000008DE873E853244A24B410182804111F1
:1006E00022C662C40008E2873E853244224C4101A2
:1006F0008280411122C666C40008E6873E853244E6
:06070000A24C41018280C1
:02000004810079
:10000000300000003100000032000000330000002A
:10001000340000003500000036000000370000000A
:10002000380000003900000061000000620000009C
:10003000630000006400000065000000660000002E
:100040002D2D2D2D2D2D2D2D2D2D2D2D2D2D2D2DE0
:100050002D2D2D2D2D2D2D2D2D0A000046494E41E3
:100060004C205A0A000000003A2000000A0000005C
:100070002D2D2D2D2D2D2D2D2D2D2D2D2D2D2D2DB0
:100080002D2D2D2D2D2D2D2D2D2D2D2D2D2D2D0AC3
:1000900000000000300000003100000032000000CD
:1000A000330000003400000035000000360000007E
:1000B0003700000038000000390000006100000037
:1000C00062000000630000006400000065000000A2
:1000D00066000000646F6E653A2000000A000000B0
:1000E00061626F757420746F207761697420666F28
:0800F0007220646F6E650A00C6
:1000F8000000008104000081080000810C000081DC
:100108001000008114000081180000811C0000818B
:100118002000008124000081280000812C0000813B
:100128003000008134000081380000813C000081EB
:1001380001000000010000000100000001000000B3
:1001480001000000010000000100000001000000A3
:100158000100000001000000010000000100000093
:100168000100000001000000010000000100000083
:100178000000000001000000020000000300000071
:100188000400000005000000060000000700000051
:1001980008000000090000000A0000000B00000031
:1001A8000C0000000D0000000E0000000F00000011
:1001B80094000081980000819C000081A0000081CB
:1001C800A4000081A8000081AC000081B00000817B
:1001D800B4000081B8000081BC000081C00000812B
:1001E800C4000081C8000081CC000081D0000081DB
:040000058000000077
:00000001FF
